:02000000102AC4
:0E00060055303C008F00AA308F000F14080008
:10001400553023009600AA30960095140000000085
:020024000800D2
:1000260023009E18182800001328210069082300C1
:040036009A00080024
:0E003A0055303C008F00AA308F000F100800D8
:1000480023009E1690309D002000901E2F2823002C
:080058001908F0002828080037
:1000600023009E183528000030282100690823004D
:040070009A000800EA
:10007400230020082100E000230021082100E100E2
:10008400230022082100E200230023082100E300CA
:10009400230024082000E700230025082000E800AE
:1000A400230026082000E900230027082000EA0096
:1000B400230028082000EB00230029082000EC007E
:1000C40023002A082000ED0023002B082000EE0066
:1000D40023002C082100DC0023002D082100DD0072
:1000E40023002E082100DE0023002F082100DF005A
:0200F400080002
:1000F6002100E601640884006508850000082000E8
:10010600EF006F08003A031998286F082100E900EC
:1001160013202100E60A6608640784000030653D66
:0C012600850000082000EF00842808007D
:100132000D302100E90030200A302100E900302092
:020142000800B3
:1001440021009901191799161916991599149801EE
:020154000800A1
:10015600FF302300A000FF30A1000030A2000030D5
:10016600A3003030A4000030A500E930A60000301E
:10017600A700FF30A800FF30A9000030AA00003019
:10018600AB00FF30AC00FF30AD000030AE000030F9
:08019600AF003A20242008000C
:10019E000B082000EF008B13230015151513951671
:1001AE0021006408230091002100650823009200BD
:1001BE002100E8011F306802031802296608840036
:1001CE0067088500000823009300013100089400A1
:1001DE0002302100E6070030E73D0A20013011070A
:1001EE00F0000030123DF10070089100710892008D
:1001FE002100E80AE12823009512210066088400F8
:10020E006708850000082300930001310008940060
:10021E000A2015112000EF1B16298B1317298B1797
:02022E000800C6
:1002300021006508F000F036F036F036F0369230E6
:10024000840084308500700884070318850A00083C
:10025000F00066088600670887007008810001309A
:10026000660786000030673D87000F306505F000A7
:100270009230840084308500700884070318850A52
:100280000008F00070088100023066078600003028
:10029000673D87006408F000F036F036F036F0363F
:1002A0009230840084308500700884070318850A22
:1002B0000008F000700881000330660786000030F7
:1002C000673D87000F306405F00092308400843071
:1002D0008500700884070318850A0008F00070087C
:1002E00081000430660786000030673D8700810189
:0202F000080004
:1002F200210066088400670885000008F000700885
:100302000319962966088400670885000008F00032
:10031200640886006508870070088100E40A0319F2
:10032200E50AE60A0319E70A7929640886006508DE
:06033200870081010800B4
:100338002100640823009100210065082300920031
:1003480015131514000000001308F0001408F1003C
:0203580008009B
:10035A00210064088400650885000008F000700820
:10036A000319C32964088400650885000008E900A8
:10037A0030202100E40A0319E50AAD290630FD0000
:08038A00FD0BC529000008006D
:1003920012001E00F003031DC929F103031DC92920
:0203A200080051
:1003A4001D203D00A50194010D309D0012309F00D9
:1003B40010309E0011309C000E303C00A0000C3028
:0C03C400A1003D00A501940103200800E9
:1003D0002200961323008C01FF3021008C000C12A8
:1003E00022000C1223008D01FF3021008D0024001B
:1003F0008D0125000D160D178D128D13F03026007E
:100400008D0027008D0123008E01DF3021008E003A
:10041000223024008E0025008E162100951308003E
:1004200020302000A0000130A100A2012008860099
:100430002108870020308100A220E821D22123005A
:100440009F15CF309B009C011E15AB2073302100FF
:10045000E4008430E500AD210330FB000830FC00EF
:100460007730FD00FD0B322AFC0B322AFB0B322ABF
:1004700080302000E5001F30E60020082100E40065
:10048000200021082100E500B930E6008330E700B4
:1004900079212B30E4008430E500AD212000A20159
:1004A0002030220203186B2A2208F000F101F035F7
:1004B000F10D2330700786000030713D870022085F
:1004C000200784000030213D850000088100413173
:1004D0008101A20A502A65082100E4002000660874
:1004E0002100E5002330E6000030E700CF20033094
:1004F000FB000830FC007730FD00FD0B7D2AFC0B73
:100500007D2AFB0B7D2A4F302100E4008430E5007A
:10051000AD212000A201203022020318AB2A2208BC
:10052000F000F101F035F10D233070078600003046
:10053000713D870020306507F0000030663DF10016
:100540002208F0070030F13D700881007108413148
:100550008100A20A8B2A203065072100E4000030C8
:100560002000663D2100E5002330E6000030E70072
:10057000CF200330FB000830FC007730FD00FD0B7E
:10058000BF2AFC0BBF2AFB0BBF2AE3302100E4008B
:100590008330E500AD212000A201203022020318A3
:1005A000ED2A2208F000F101F035F10D233070073B
:1005B00086000030713D870040306507F000003054
:1005C000663DF1002208F0070030F13D700881001F
:1005D000710841318100A20ACD2A4030650721000F
:1005E000E40000302000663D2100E5002330E600F5
:1005F0000030E700CF200330FB000830FC007730EC
:10060000FD00FD0B012BFC0B012BFB0B012B07301D
:100610002100E4008430E500AD212000A20120305B
:10062000220203182F2B2208F000F101F035F10D02
:100630002330700786000030713D87006030650709
:10064000F0000030663DF1002208F0070030F13D77
:1006500070088100710841318100A20A0F2B6030BF
:1006600065072100E40000302000663D2100E50020
:100670002330E6000030E700CF200330FB000830D5
:10068000FC007730FD00FD0B432BFC0B432BFB0BD9
:10069000432B8C302100E4008330E500AD212000A5
:1006A000A2018030220203188B2B65082100E40090
:1006B000200066082100E5009C2170082000E3006E
:1006C0007108E400E50A0319E60A0D30FD00FD0B90
:1006D000672B63082100E400200064082100E50086
:1006E000A030E6000030E7001821A030E400003020
:1006F000E5007B2099200230FB000430FC00BA307A
:10070000FD00FD0B812BFC0B812BFB0B812B0000D3
:080710002000A20A512B8B2BE3
:100718002034523465346C3465346334743475343D
:1007280072346534203464346534203431343234DE
:100738003834203462347934743465347334203472
:10074800E03420347034613472347434693472346F
:1007580020346434653420343034783431344634C9
:0A076800383430340D340A34003404
:100772004134423443343134323433343434353412
:1007820036344434453446344734483430343134D2
:10079200323433343434353436343734383439340B
:1007A2004134423443344434453446344734483483
:1007B20049344A344B344C344D344E344F34503433
:0407C200513400347A
:1007C6002034453463347234693474342034333419
:1007D6003234203464346134743461342034E03487
:1007E6002034703461347234743469347234203491
:1007F6006434653420343034783431344634433408
:0808060030340D340A340034D3
:10080E0020344534633472346934743420343334D0
:10081E003234203464346134743461342034E0343E
:10082E002034703461347234743469347234203448
:10083E0064346534203430347834313446344534BD
:08084E0030340D340A3400348B
:100856002034453463347234693474342034333488
:100866003234203464346134743461342034E034F6
:100876002034703461347234743469347234203400
:100886006434653420343034783431344634383482
:0808960030340D340A34003443
:10089E002034453463347234693474342034333440
:1008AE003234203464346134743461342034E034AE
:1008BE0020347034613472347434693472342034B8
:1008CE006434653420343034783431344634413431
:0808DE0030340D340A340034FB
:1008E6000D340A34203446344C34413453344834BD
:1008F6002034543445345334543420342834483462
:10090600453446342934203431343634463431348F
:0E09160036343134393420340D340A34003490
:100924003034313432343334343435343634373487
:10093400383439344134423443344434453446340D
:020000040001F9
:06000E00E408831C1F3F03
:00000001FF
